S123A1007EA13C0000000000426567416464723A2004456E64416464723A2004537461726F
S123A12074207461706520616E6420707265737320656E746572044F4B0D0A0486F0970237
S123A140CEA108BDC009BDC01EFFA104BDC021CEA112BDC009BDC01EFFA106BDC021CEA1CC
S123A1601CBDC009BD7FEB810D2620BDC021BDA18EFEA104A600BDA1B508BCA10623F5BD18
S123A180A18E7F8060CEA137BDC0097EC000CE0800C600F78060BDA1F5C601F78060BDA101
S123A1A0FB0926EDC600F78060BDA1F5C601F78060BDA1F539C608F7A103C600F78060BDA7
S123A1C0A1F5C601F78060BDA1F5442512C600F78060BDA1F5C601F78060BDA1F52010C6A2
S123A1E000F78060BDA1F5C601F78060BDA1FB7AA10326D639C6325A26FD39C6645A26FD92
S104A2003920
S9030000FC
